:020000040800F2
:1000000000040010390C0008B92D0008BF2D0008AD
:10001000C52D0008CB2D0008D12D000800000000E0
:10002000000000000000000000000000DD2D0008BE
:10003000D72D000800000000E32D0008E92D00087E
:10004000EF2D0008EF2D0008EF2D0008EF2D000820
:10005000EF2D0008EF2D0008EF2D0008EF2D000810
:10006000EF2D0008EF2D0008EF2D0008EF2D000800
:10007000EF2D0008EF2D0008EF2D0008EF2D0008F0
:10008000EF2D0008EF2D0008EF2D0008EF2D0008E0
:1000900019080008EF2D0008EF2D0008EF2D0008CB
:1000A000EF2D0008EF2D0008EF2D0008EF2D0008C0
:1000B000EF2D0008EF2D0008EF2D0008EF2D0008B0
:1000C000EF2D0008EF2D0008EF2D0008EF2D0008A0
:1000D000EF2D0008EF2D0008EF2D0008EF2D000890
:1000E000EF2D0008EF2D0008EF2D0008EF2D000880
:1000F000EF2D0008EF2D0008EF2D0008EF2D000870
:10010000EF2D0008EF2D0008EF2D0008EF2D00085F
:10011000EF2D0008EF2D0008EF2D0008EF2D00084F
:10012000EF2D0008EF2D0008EF2D0008EF2D00083F
:10013000EF2D0008EF2D0008EF2D0008EF2D00082F
:10014000EF2D0008EF2D0008EF2D0008EF2D00081F
:10015000EF2D0008EF2D0008EF2D0008EF2D00080F
:10016000EF2D0008EF2D0008EF2D0008EF2D0008FF
:10017000EF2D0008EF2D0008EF2D0008EF2D0008EF
:10018000EF2D0008EF2D0008102808B500D9FEE774
:10019000034B53F8200001F011F980B208BD00BFF5
:1001A000C0320008102800D9FEE7024B53F82000A7
:1001B00001F0F4B8C0320008034A9068D36851696E
:1001C0000344194402F043BD803F000808B502F023
:1001D0005BFD00F02BFE054BD9689868890800F09C
:1001E0002DFEBDE8084000F037BE00BF803F00088C
:1001F00000B599B001A800F019FF0B49019A0B4B0B
:10020000B2FBF3F30B600A4B1A600A4AD36843F05F
:100210008073D360084A1368002043F00103136021
:1002200019B05DF804FB00BF2001002040420F0020
:100230001C010020F0ED00E0001000E009490A4B2D
:100240000A6830B51D6800230C68A21A1344B3FB7A
:10025000F5F2824204D2801A05FB12332246F3E7FC
:10026000002030BD041000E020010020034B18687E
:10027000034B1B68B0FBF3F0704700BF041000E0B5
:10028000200100202DE9F04782460D4601B9FEE726
:10029000CAF800104FF000082B795FFA88F7BB42CC
:1002A00049D918247C432E68244A3359934206EBDB
:1002B00004091AD007D8B3F1904F10D0A2F580628C
:1002C00093420FD029E01E4A934214D002F5806277
:1002D000934213D0A2F50062934209D01DE04FF47F
:1002E00000300DE04FF480200AE04FF4002007E0DA
:1002F0004FF4801004E04FF4001001E04FF4800050
:10030000012101F00FF8D9F810203AB13059B9F8AD
:100310000410D2B202F0CEFD00E0FEE7305909F140
:10032000040102F077FDDAF80000394602F0D7FC4C
:1003300008F10108B0E70020BDE8F0870008004898
:1003400000100048074B1A681AB9EFF310820649EB
:100350000A604FF0010080F310881A6801321A60B9
:10036000002070472801002024010020074B186856
:1003700038B10138186038B9054B1B6883F3108811
:1003800070474FF0FF307047002070472801002071
:100390002401002007B500F097FC00F013FD0021B8
:1003A0001F4800F027FE4FF4407000F0E3FD0420EA
:1003B00000F02AFEFFF71CFF1A48012100F0B2FFEF
:1003C0001948012100F0C6FF0121184800F0B6FFCE
:1003D000684602F05BFD01238DF80730694640F264
:1003E000FF734FF09040009302F014FD4FF6FF733F
:1003F00069460F48009302F00DFD69460D4802F072
:1004000009FD69460C4802F005FD69460B4802F0FB
:1004100001FD0B48694602F0FDFC03B05DF804FBEA
:100420000000000857007E3137C8FE32017807000F
:100430000004004800080048000C00480010004874
:100440000014004808B5FFF77DFF002001F0A6FF6B
:10045000012001F0A3FF022001F0A0FFBFF34F8FA6
:100460000449054BCA6802F4E0621343CB60BFF352
:100470004F8FFEE700ED00E00400FA05034B10B1DA
:1004800001221A7000E0187000207047D502002089
:10049000F7B5194D03272F60684602F0F7FC0024DA
:1004A0004FF48053694601264FF0904000938DF839
:1004B00005708DF8046002278DF8064002F0AAFC52
:1004C000322002F0E5FB2F600520FFF7B7FE0B4B53
:1004D0002C6069461C604FF090408DF8047002F06B
:1004E00099FC204600F018FF4FF40000314600F060
:1004F00031FF204603B0F0BD405C0040445C00404A
:1005000073B5064600B9FEE701B9FEE7244B1D7836
:10051000002D40D10122234C1A70234B61602360CF
:10052000FFF7B6FF6068214B08301C6000F02CFD1F
:100530004FF4C053009303238DF805304FF09040E3
:10054000022369468DF804308DF806508DF8075067
:1005500002F060FC4FF090400B210E2202F0AAFC4A
:100560004FF090400C210E2202F0A4FC6168C86894
:1005700010B1103102F04EFC002000F0CDFE4FF41F
:100580000000012100F0E6FE01F0AAFB01F0FEFCF4
:100590003460002001E04FF0FF3002B070BD00BFBA
:1005A000D40200202C010020045936173401002009
:1005B00008B50C4B186898B102680B4B9A4201D0F1
:1005C000002008BD4368D86830B1198A02F068FC81
:1005D000431E5842584108BD044B1878C0B208BDAC
:1005E00008BD00BF3401002004593617D602002090
:1005F00008B50A4B1B682BB11A68094B9A4203D005
:10060000002008BD184608BDC0B2FFF7D1FF08B1F1
:10061000044B187800F0010008BD00BF3401002031
:1006200004593617D5020020014B01221A70704779
:10063000D6020020014B00221A707047D60200201B
:1006400010B5044B04689C4200D0FEE70261C16013
:1006500010BD00BF00BB00AA10B5044B04689C424B
:1006600000D0FEE78261416110BD00BF00BB00AA5F
:1006700038B502680F4B9A4204460D4600D0FEE79B
:100680008068FFF7B5FFA0B1FFF75CFE636858789C
:1006900002F096FCB0F5405F07D03E2D05D96368A7
:1006A0004FF44051587802F069FCBDE83840FFF73C
:1006B0005DBE38BD00BB00AA02680B4B9A4210B564
:1006C000044600D0FEE78068FFF792FF50B16368F0
:1006D000987802F06CFC302804D02046BDE8104029
:1006E00002F036BB10BD00BF00BB00AA084B10B51E
:1006F0001C68084B22689A4200D0FEE7A068FFF70A
:1007000077FF20B12046BDE8104002F021BB10BDAC
:10071000DC01002000BB00AA1E4B30B51C681E4B3C
:1007200022689A4285B000D0FEE76368587801F0ED
:100730001DFC63680546587801F0DAFB402D2A4617
:1007400028BF4022014692B204F11C0002F0DDFBFA
:10075000E56815B96368587815E000238DF80D3009
:100760000DF10D03009320690DF10E0304F11D013D
:100770003F22A847BDF80E303E2B6368587802D957
:100780004FF4405101E04FF4005102F0F7FB05B087
:1007900030BD00BFDC01002000BB00AA2DE9F04104
:1007A0000E469046074600B9FEE701B9FEE7124B38
:1007B0001C78E4B9114D01221A7021462846A42262
:1007C00002F0E4F90E4B0F4A0F4985E848010F4B40
:1007D0001D60B378013B204642F8231073780C4A21
:1007E0000C49013B42F823103D60BDE8F0814FF019
:1007F000FF30BDE8F08100BFD702002038010020A3
:1008000000BB00AA00000020ED060008DC0100206B
:100810001C0000201907000870B52D4D2D4C2B68C9
:100820002D4E9BB22380228833881340190401D5B2
:1008300001F070FA2288338813405A0505D54FF627
:10084000FF332B60254B5B689847228831880A402C
:10085000930444BF4DF6FF732B6023880B40D804EC
:1008600005D54EF6FF732B60002000F083F8228838
:100870003388134019050DD5194B1B7813B100F0BF
:1008800047F802E0022000F075F84FF2FF732B608A
:10089000FFF7D0FE2288338813409A0509D54FF61A
:1008A000FF53104A2B6013780133DBB21370FFF74C
:1008B000BBFE228833881340DB0507D54FF6FF6364
:1008C0002B600720BDE8704000F054B870BD00BF39
:1008D000445C0040500500205A03002038000020EE
:1008E000C0000020D8020020064B074901221A60F0
:1008F000064A0020186010604FF4E0520A801A6027
:10090000704700BF405C00405A030020445C004038
:10091000074A13689BB243F00803136013689BB245
:1009200043F004031360034B03221A60704700BFB7
:10093000405C0040E0010020044B9A7A044B0AB16D
:10094000052200E001221A60704700BF3403002036
:10095000E001002010B5064C22684FF6FB731340EF
:100960002360FFF7E9FF4FF43F43236010BD00BF52
:10097000405C004010B51E4C072818BF207023783B
:10098000052B32D8DFE803F003060A0E1621FFF725
:10099000E1FF2AE0FFF7DEFF042327E00223637074
:1009A000032323E06378013BDBB263706378F3B920
:1009B000042217E00F4A13689BB243F01003136040
:1009C000052323700A23637010BD6378013BDBB2FB
:1009D000637063785BB9074A11684FF6EF730B4099
:1009E00013600622024B1A7010BD0623237010BD3F
:1009F00058050020405C0040014B04221A607047FB
:100A0000E001002010B5034C236813B19847002380
:100A1000236010BDE401002010B5134B1B681A7849
:100A200002F07F02012A02D0212A0CD00FE05A796D
:100A30006AB906280BD19A78212A02D0222A08D036
:100A400005E00A4A08E05A790AB9032803D00220CF
:100A500010BD074A00E0074A9A6100245C822046E4
:100A60009047204610BD00BF54030020C90A00086B
:100A7000D50A0008790A000820B9034B1B68012237
:100A80001A82704701487047540300202803002051
:100A9000054B1B68DB78042B04D8044901EBC30128
:100AA00000F0C8BF00207047540300200802002057
:100AB000014900F0BFBF00BFE8010020014900F07C
:100AC000B9BF00BF00020020014900F0B3BF00BF62
:100AD000F0010020014900F0ADBF00BFF801002087
:100AE000254B1B6810B500249C72DC725C7220469A
:100AF00001F0C6F920464FF4007102F018FA2046C2
:100B0000402101F0C5F91021204602F01EFA2046CE
:100B100002F085FA2046202101F0CAF9174B204641
:100B200093F82C1001F002FA204602F065FA012039
:100B30004FF4C06102F0FBF90120602101F0A8F937
:100B40000120402101F0E4F90120202102F0FDF90B
:100B50000120802101F0ACF90120402101F0E6F9EB
:100B600001204FF4405102F009FA204601F068F8E4
:100B7000034B01221A6010BD5403002038000020EE
:100B8000E0010020054B10B51B6800249C72FFF7A4
:100B9000ABFE01F0FBF9024B1C6010BD54030020BA
:100BA000E0010020054B1B68987A10B1044B052228
:100BB0001A60003018BF0120FFF760BC540300200A
:100BC000E0010020084B1A68137803F07F03212B03
:100BD00008D1537933B90B2804D1D178034A184688
:100BE0001160704702207047540300202803002042
:100BF000014B18609980704700020020014B19607A
:100C00009A807047E801002003289FBF034B43F8F8
:100C1000301003EBC0039A80704700BF0802002029
:100C2000014B186099807047F0010020014B18605B
:100C300099807047F8010020194CA246194A1A48B9
:100C4000536A43F4E0235362184B596841F0404122
:100C50005960D96841F00071D960D96841F080715C
:100C6000D960D2F88830124943F47003C2F8883052
:100C7000104A121A01F0F0FE0F48104A0021121A11
:100C800001F084FF0E480F4A0021121A01F07EFF86
:100C9000A5214FF47072204601F078FF01F0DCF9D5
:100CA0000000001000ED00E00000002030EF00E048
:100CB000403400081C0100201C0100205A050020BF
:100CC0000004001000040010394AD2F8883043F4C0
:100CD0007003C2F88830374B1A6842F001021A607C
:100CE0005968354A0A405A601A6822F0847222F420
:100CF00080321A601A6822F480221A605A6822F43C
:100D0000FE025A60DA6A22F00F02DA62196B2B4A8D
:100D100082B00A401A6300229A60009201921A6817
:100D200042F480321A601A6802F400320192009A8A
:100D300001320092019A1AB9009AB2F5A04FF2D18D
:100D40001A6812F4003218BF01220192019A012A96
:100D500005D0174B4FF000629A6002B07047184AF6
:100D6000122111605A685A605A685A605A6842F4EF
:100D700080625A605A6822F47C125A605A6842F4BF
:100D8000E8125A601A6842F080721A601968094ABB
:100D90008901FBD5516821F003015160516841F090
:100DA000020151605A6802F00C02082AFAD1D0E719
:100DB00000ED00E0001002400CC07FF8CCFC00FF0A
:100DC00000200240144A1549536803F00C03042B19
:100DD00010B501D0082B01D0114B12E053685068B8
:100DE000C00349BFD06A0F480D4C00F00F00C3F399
:100DF000834348BF013003F1020348BFB4FBF0F066
:100E000043430B605368084AC3F30313D25C0B6877
:100E1000D3400B6010BD00BF001002408C000020CA
:100E200000127A0000093D00C3000020024A9368C6
:100E300043F00103936070470030024000EB8101F2
:100E40008842044B03D050F8042B1A60F8E7186866
:100E5000704700BF00300240014B1868704700BF68
:100E600000300240034A136823F003031843106064
:100E7000704700BF00200240044B1A6810B142F0D6
:100E8000100201E022F010021A60704700200240B8
:100E9000044B1A69120641BF034A5A6002F18832B4
:100EA0005A6070470020024023016745024A1369D7
:100EB00043F080031361704700200240084BDA685A
:100EC000D10709D4DA68D20608D4DB6813F0040F1E
:100ED00014BF032004207047012070470220704790
:100EE0000020024038B505464FF4302001F081FF64
:100EF000042811D1094C236943F002032361656181
:100F0000236943F0400323614FF4302001F071FF67
:100F1000236923F00203236138BD00BF0020024093
:100F200073B5002306464FF430200D46019301F0BF
:100F300060FF042819D10E4C236943F0010323619B
:100F4000ABB233804FF4302001F053FF042808D1B6
:100F500002360196019B2D0C1D804FF4302001F0CC
:100F600048FF236923F00103236102B070BD00BF75
:100F70000020024040F0BF60024B40F40030D860D7
:100F8000704700BF00ED00E0C278037810B50AB3E7
:100F9000164AD4684278E443C4F30224C4F104013D
:100FA00002FA01F10F22E240847822400A4303F161
:100FB000604303F561431201D2B283F80023037842
:100FC0000122590903F01F0302FA03F3084A42F809
:100FD000213010BD5A09012103F01F03994002F18D
:100FE0002003034A42F8231010BD00BF00ED00E0CB
:100FF00000E100E021F0604121F07F01014B084356
:101000009860704700ED00E0044B1A6804280CBF9C
:1010100042F0040222F004021A60704710E000E07F
:10102000014B1860704700BF20000E422DE9F041CF
:101030009B4F7B6803F00C03042B05D0082B06D0D4
:10104000984A0260B3B916E0964B036012E07B68E1
:101050007968C3F383439A1CCB0349BFFB6A924B65
:10106000904903F00F0344BF0133B1FBF3F3534343
:10107000036000E000237A688C4EDFF834C2C2F3CC
:101080000312B45C0268E4B222FA04F141607D68A4
:10109000C5F30225755D21FA05FEC0F808E07D68FC
:1010A000C5F3C225755DEDB2E940C160FE6AC6F3C5
:1010B000041808F00F0618F0100F3CF81660E04610
:1010C000B6B204D01EB1B3FBF6F6066100E00261D1
:1010D000FE6AC6F3442C0CF00F061CF0100F38F813
:1010E0001660B6B204D01EB1B3FBF6F6466100E05E
:1010F00042613E6BF6065ABF6A4E866182613E6B64
:10110000B6065ABF674EC661C2613E6B76065ABFCD
:10111000644E066202623E6BF60506D59A4204D121
:10112000A54202D15600466200E041623E6BF604E1
:1011300006D59A4204D1A54202D15600866200E04B
:1011400081623E6BB60506D59A4204D1A54202D112
:101150005600C66200E0C1623E6B760506D59A4233
:1011600004D1A54202D15600C66400E0C1643E6BC2
:10117000360506D59A4204D1A54202D1560006652D
:1011800000E001653E6BB60406D59A4204D1A54243
:1011900002D15600466500E001653E6B360406D577
:1011A0009A4204D1A54202D15300836500E08165D3
:1011B0003C6B3B4BA40701D1816315E0196B01F037
:1011C0000301012901D182630EE0196B01F00301D3
:1011D000022902D14FF4004305E01B6B03F0030327
:1011E000032B01D12F4B8363396B2D4B11F4403FFF
:1011F00002D1C0F83CE018E0196B01F44031B1F5C0
:10120000803F01D1C26310E0196B01F44031B1F5A8
:10121000003F02D14FF4004306E01B6B03F4403360
:10122000B3F5403F01D11F4BC363396B1C4B11F425
:10123000402F02D1C0F840E018E0196B01F44021C2
:10124000B1F5802F01D1026410E0196B01F4402147
:10125000B1F5002F02D14FF4004306E01B6B03F4FD
:101260004023B3F5402F01D10E4B0364396B0C4B77
:1012700011F4401F02D1C0F844E023E0196B01F4DF
:101280004011B1F5801F01D142641BE0196B01F4DC
:101290004011B1F5001F0DD14FF4004311E000BF24
:1012A0000010024000127A0000093D00D300002027
:1012B000A00000201B6B03F44013B3F5401F01D1C5
:1012C000134B4364396B134B11F4400F03D1C0F837
:1012D00048E0BDE8F081196B01F44001B1F5800FE1
:1012E00002D18264BDE8F0811A6B02F44002B2F5CB
:1012F000000F02D14FF4004306E01B6B03F44003E0
:10130000B3F5400F01D1024B8364BDE8F08100BF0B
:1013100000127A0000100240014B1860704700BFB5
:10132000D8004242044B5A6909B1104301E022EA55
:1013300000005861704700BF00100240044B9A69DA
:1013400009B1104301E022EA00009861704700BF34
:1013500000100240044BDA6909B1104301E022EAAF
:101360000000D861704700BF00100240044BDA68EB
:1013700009B1104301E022EA0000D860704700BFC5
:1013800000100240044B1A6909B1104301E022EA3F
:1013900000001861704700BF0010024082B00023B7
:1013A0000193054B0193019B03EB80000190019B8E
:1013B000196002B0704700BF5028004082B000237F
:1013C0000193054B0193019B03EB80000190019B6E
:1013D000186802B0704700BF502800400549064A0F
:1013E000CB68024042F0800203F0800363EA02030C
:1013F000CB607047002800407FFF010010B5064C0D
:1014000018B9236801221A8210BD044B1B681B689F
:10141000984720680A3010BD540300205003002074
:1014200010B5064C18B9236801221A8210BD044B6E
:101430001B689B68984720680C3010BD540300203F
:101440005003002010B5214A18B9136802221A82ED
:1014500010BD1F48146800230380217811F07F011C
:1014600002460ED1637A990644BF0221017013F03F
:10147000400F037814BF43F0010323F0010303700E
:101480001CE0012921D002291ED1637913F0800FBD
:1014900003F00F034FEA830303F1804303F5B843DE
:1014A0001B6806D003F03003102B07D10123137003
:1014B00004E003F44053B3F5805FF7D0054B1B689D
:1014C0001B699847024810BD184610BD5403002000
:1014D00052050020500300202DE9F843234FDFF888
:1014E000A0803D682B8A2E7ABBB9042E15D12048E6
:1014F0000278012A0CD11F4A11681F4A89B20A4496
:101500005200138053803022A8F80020037029E095
:101510001023A8F80030072624E0AC8AA34294BF29
:10152000042602269C4228BF1C462046AB699847E9
:101530008146002000F0CCFC22460146484601F0DE
:10154000CCFC0020214600F0E3FC2B8A1B1B2B82E5
:101550006B8A23446B823023A8F80030074B4FF48A
:1015600040521A803B681E72BDE8F8835403002085
:10157000D9020020505C00400230002054050020B9
:101580005605002037B5694C23685A78062A13D1CE
:101590001A78520678D19A78654B012A02D11B68D5
:1015A000DB6968E0022A02D11B681B6A63E0032A38
:1015B0006AD11B685B6A5EE0002A3DD15988002928
:1015C00062D15A6822F47F42B2F5003F5CD11A78AA
:1015D00012F07F0204D19B88002B00F09F8053E023
:1015E000012A0CD1524A5879126892699047002812
:1015F0004AD123689B7A002B40F0908044E0022A75
:1016000042D15A794B4802F00F010BB29B0003F113
:10161000804303F5B84300781B6812F0800F14BFB5
:1016200003F0300303F4405381422DD212F0700FC7
:101630002AD1002B72D127E0082A03D11B785B0640
:101640006ED021E00A2A1FD11A7802F07F02012A07
:101650001AD19A7AC2B15988B1B95A6822F47F4234
:10166000B2F5803F10D1324A58791268926990479A
:10167000002857D008E03BB12268002555829361CD
:101680002846984728460CE0294B22681B6850786A
:101690001B699847032804D1244B1B6809221A723E
:1016A00042E023681A8A4FF6FF718A4202D109226A
:1016B0001A7239E0022800D012B908221A7233E0F7
:1016C00093F90010002922DAD98801910198184C69
:1016D000824202D9019A1A8212E08A4210D221680B
:1016E00091F82C00824203D2134A0021117007E0C6
:1016F00092FBF0F100FB112212B90F4A0121117087
:10170000226892F82C209A82FFF7E6FE0CE0032272
:101710001A720A4B4FF440521A8005E0084BABE7AF
:10172000084BA9E7084BA7E703B030BD54030020DE
:1017300030030020C1000020D90200205405002001
:1017400045140008FD1300082114000810B50A4BC9
:101750000A491B684978DA7891420AD3997841B9E5
:101760009C8834B99A72064B1B685B689847204680
:1017700010BD022010BD00BF54030020C100002096
:101780005003002038B50E4A0E4D12682B6892693E
:101790005879D97890472B689A7A7AB170B91A79C2
:1017A00062B99C7854B9084B1B68DB6898472B6872
:1017B0005A79DA72DA781A73204638BD022038BDB9
:1017C00030030020540300205003002038B5314B73
:1017D0001B68187810F07F0004D15A7A22F020029A
:1017E0005A7238BD022853D15A88002A51D11A7929
:1017F000002A4ED15979284D21F08000840004F14F
:10180000804202F5B8422D78126811F0800F14BFA3
:1018100002F0300202F44052A84239D2002A37D0F6
:101820009B7A002B34D004F1804404F5B8440A06B6
:1018300023680CD503F03003102B23D1C4B220460B
:1018400001F010FC2046302101F07FFB1AE003F488
:101850004053B3F5805F15D128B9104B93F82C1085
:1018600000F064FB01E001F0EAFB236823F480430D
:1018700023F070039BB283F4405343F4004343F0DE
:1018800080032360064B1B685B699847002038BDC6
:10189000022038BD54030020C10000203800002081
:1018A0005003002038B51F4B1F4D18682D78417923
:1018B00021F08004A30003F1804202F5B84211F048
:1018C000800F126814BF02F0300202F44052AC42A2
:1018D00025D244881CBB12B3827A02B303F1804341
:1018E00003F5B84309061A684BBF22F4E04222F41C
:1018F000804222F0400222F070024BBF92B292B2BC
:1019000082F0100282F4805242F4004242F08002DF
:101910001A60064B1B689B699847002038BD02205F
:1019200038BD00BF54030020C10000205003002038
:1019300008B5064B1A68537A43F020035372044BE0
:101940001B68DB699847002008BD00BF54030020D6
:101950005003002038B5324D2B681A785C7812F0AD
:101960007F0237D1092C02D1FFF7F0FE41E0052CB0
:101970000FD193F90320002A01DA08234CE09A786A
:10198000002AFAD19A88002AF7D19B7A002B34D00A
:10199000F3E7032C10D1DA78012A07D0214B1B681A
:1019A00020465B699847032825D134E09B88002BAB
:1019B000F4D1FFF7BDFF1CE0012CEFD1DA78012A4A
:1019C000ECD19A88002AE9D15B7A9B06E6D5FFF72D
:1019D000FDFE0EE0012A04D10B2CDFD1FFF7D2FE71
:1019E00007E0022ADAD1012CF1D0032CD6D1FFF77F
:1019F00059FF10B1D2E70028BFD10B4B1A680B4B2F
:101A000092B213445B0000221A805A80084B3022A5
:101A10001A80062300E009232A68137238BD00BF2C
:101A20005403002030030020505C004002300020AE
:101A300056050020054B10B51C68628A18B98B88C2
:101A40009B1A238210BD0868104410BD5403002067
:101A500008B50C4B002093F82C1000F067FA0A4BE5
:101A60001B68187A082801BF084B4FF480521A806F
:101A7000074B04BF10221A80A0F1090358425841B5
:101A800008BD00BF3800002054030020540500208A
:101A90005605002090B583B000AF0123FB80304B8A
:101AA0001B689BB21A462F4B13445B001B689BB20A
:101AB0005B0003F1804303F5C0433B602A4B1B6886
:101AC0001B7A092B37D0284B1A683B68591C3960A0
:101AD0001B781370244B1A683B68591C39601B78BB
:101AE00053703A68FB885B0013443B601E4B1C68D4
:101AF0003B689A1C3A601B88184601F0C6FA0346F8
:101B000063803A68FB885B0013443B60164B1C689B
:101B10003B689A1C3A601B88184601F0B6FA0346E7
:101B2000A3803A68FB885B0013443B600E4B1B6844
:101B30003A681288DA800C4B1B6801221A720A4B31
:101B40001B68DB88002B02D1FFF704FF01E0FFF7E1
:101B500019FDFFF77DFF034618460C37BD4690BDC3
:101B6000505C00400430002054030020F8B52E4D96
:101B70002C68237A022B4FD0042B4DD0032B01D09D
:101B8000052B41D1A169238AA9B1A3B1A68A9E429E
:101B900028BF1E4630468847238A9B1B2382638AC0
:101BA000334407466382002000F0A2F93246014622
:101BB000384601F0AAF9238A53B11C4B00204FF498
:101BC000405201461A8000F0A3F9194B30221A80C6
:101BD000A38A228A93422B6802D803221A7210E049
:101BE00012B105221A720CE006211972114B196804
:101BF000114B89B20B445B001A805A800C4B302287
:101C00001A802B681B7A08E0072B05D10B4B1B6849
:101C1000DB689847082300E008232A681372BDE8B0
:101C2000F840FFF715BF00BF540300205405002003
:101C300056050020505C0040023000203003002098
:101C400070B50D4B1D780022AA4210D202F18053CC
:101C500003F5B8539B0042F400441E6840F60F7130
:101C600044F080043140214319600132ECE7034B1A
:101C700040F08000186070BDC10000204C5C004046
:101C800010B5144C23681A7A022A01D0042A04D110
:101C9000FFF722FC23681B7A15E0062A12D15A7836
:101CA000052A09D11A78520606D1D878FFF7C8FF5D
:101CB000094B1B681B6A9847084B1B689B68984731
:101CC000082300E0082322681372BDE81040FFF7E4
:101CD000BFBE00BF5403002050030020300300208B
:101CE000064A074B136002221A72064A064B13601B
:101CF000064A074911601B68184700BF54030020BB
:101D0000340300203003002038000020500300205E
:101D10006800002073B50023ADF80630504B514ADF
:101D20001B6899B21B04118040F1978013884E4CB8
:101D300003F00F032370002B61D14C4C4C4D2368F2
:101D40004C4E9BB22B802B8803F0300333802B88C2
:101D500003F440532B8021684BF6BF730B4083F490
:101D6000005383F0200343F4004343F080032360D7
:101D70001388D80607D4226848F60F7313402360EF
:101D8000FFF77EFF1BE023689BB2ADF80630BDF87D
:101D90000630190507D5226840F68F73134023607B
:101DA000FFF778FE0BE0BDF806301BB2002BB5DA6A
:101DB000226840F68F7313402360FFF7D7FE226836
:101DC0004BF6BF7313402A88D2042A8848BF83F495
:101DD00080539404328848BF83F40053D00632887D
:101DE00048BF83F01003910648BF83F0200343F4FB
:101DF000004343F080031D4A9BB213602DE09A001C
:101E000002F1804202F5B842116889B2ADF80610BD
:101E1000BDF8061009B2002909DA106840F68F7182
:101E200001401160013B144A52F823309847BDF835
:101E300006301A067FF572AF2278930003F18043D3
:101E400003F5B84348F60F71186801401960013A6C
:101E50000A4B53F82230984760E702B070BD00BFCC
:101E6000445C0040500500205C030020005C004002
:101E700054050020560500201C0000200000002012
:101E80004FF6F873014A034013607047505C0040FE
:101E9000064B1B689BB203EBC00000F1005000F53D
:101EA000405049084000490001607047505C0040C4
:101EB000054B1B689BB203EBC000044B034449086D
:101EC0005B00490019607047505C004004300020FE
:101ED000064B1B689BB203EBC00000F1005000F5FD
:101EE00040504000006880B2704700BF505C004026
:101EF000054B1B689BB203EBC000044B03445B0023
:101F0000186880B2704700BF505C00400430002069
:101F1000044B1B689BB203EBC000034B03445B0004
:101F200019607047505C0040023000200D4B1B6868
:101F30009BB203EBC0000C4B3E2903444FEA430223
:101F400009D94B09C80604BF03F1FF339BB29B02BA
:101F500043F4004304E04B08C90748BF01339B0228
:101F600013607047505C004006300020054B1B6832
:101F70009BB203EBC000044B03445B001868C0F342
:101F800009007047505C004006300020044B054AB1
:101F9000002018604FF43F431380034A13607047DA
:101FA000445C00405A030020405C00401B4B10B5CD
:101FB0009C6823685B0C5B04B3F1005F02D0B3F153
:101FC000805F24D1FEF772FF4FF0FF300121FFF751
:101FD000CDF94FF0FF300121FFF7D4F94FF0FF307A
:101FE0000021FFF7C3F94FF0FF300021FFF7CAF9D6
:101FF0000B4A0023136053600A4A636813600A4A5D
:102000001360226882F30888BDE810401847074B28
:102010000C221A70064B00221A7010BD803F000877
:10202000405C00406003002064030020680300203F
:10203000DB02002008B5064B064918683F2201F074
:10204000C0F810B1034800F0F3F9012008BD00BF4B
:102050006C030020DD0200202DE9F047FEF79AF91D
:1020600000F0CEF801F0D4F80020FEF7A1FA544CAD
:10207000207001F0D4F80128054607D14FF47A709A
:1020800000F006FE4F4B1D7001F0DDF82378012BA8
:1020900004D04C4B1B785A1E534253414A4A4B4F73
:1020A0001370012BDFF8409109D100F0A9F8454BDE
:1020B0001B78012B0CBF002307233B7002E0012398
:1020C00089F80030FEF7D2F800248046404600F040
:1020D000EAFD99F80030012B8044044401D1FFF758
:1020E00065FF3B783A4E3B4D092B2ED8DFE803F0D5
:1020F000050A2D2D2D0517232D0541F28833336058
:10210000642210E041F288333360334B64221A605A
:1021100040F6C4132B60314B32221A601EE040F6A9
:10212000C413336032222C4B00201A6000F036F9C1
:1021300000232B6012E04FF0000A5046C6F800A0C2
:1021400000F024F9C5F800A008E041F288323260BE
:1021500021492A60214A64230B601360306828B14A
:102160001D4B2246196800F095FF18B1002000F0C1
:102170000DF901E000F012F9286848B1174B22462A
:10218000196800F087FF18B1002000F0FFF802E0A6
:10219000002000F003F9124B9C4209D8114B9C42DD
:1021A00007D93B78072B04D1012389F8003000E0E0
:1021B0000024FFF73FFF002000F0E6FB86E700BFAA
:1021C0001C030020DC020020DA020020680300204B
:1021D000980000209C000020900000209400002027
:1021E00080F0FA02808D5B00DB0200200A46034982
:1021F00003460868194600F0B6BF00BF6C03002014
:1022000013B5154C237823BB0120FEF735FE0220C1
:10221000FEF728FE114800F0B1F800F063F800F076
:1022200091F80F496846FEF76BF901A80D49009A2D
:10223000FEF7B4FA00B1FEE70B480C49019A00F032
:1022400017F800B1FEE740200121FFF76BF80123EA
:10225000237002B010BD00BF1D030020983300089A
:1022600030330008DC3300086C0300200033000822
:10227000F8B51646074600B9FEE701B9FEE78B69D7
:1022800003B9FEE74B6903B9FEE70D4C0025616019
:102290002260104684F8475022460A4998476368EE
:1022A00020681B693F219847636884F8875030464F
:1022B0009B690549224698473C602846F8BD00BF07
:1022C0002802002017310008C3300008032800D975
:1022D000FEE7034B89B233F81000FDF763BF00BF80
:1022E000A033000810B5124C88B001A800F00DFD15
:1022F00001A9A01C182200F0B5FF0E49032200F02E
:10230000B1FF02200C491222FEF77EFC2146032079
:102310003822FEF779FC002008490422FEF774FCFD
:10232000012007491C22FEF76FFC002008B010BDF9
:10233000E3000020A6330008AA330008D8330008C1
:10234000BC33000810B50A4C292221460120FEF7B3
:1023500055FC08481221FEF74BFC04F1120009213C
:10236000FEF75EFC04482421FEF760FC002010BD4F
:102370001534000803340008DF330008014600B9B3
:10238000FEE70148FDF77EBFB0020020024BC1B25C
:10239000186800F08EBC00BFB0020020024BC1B232
:1023A000186800F09CBC00BFB002002030B10128CA
:1023B00007D1054B98685B6818447047024B586812
:1023C00070470020704700BF74030020034B1B7848
:1023D0000BB9FDF7FBBE0020704700BF0F050020C2
:1023E0002DE9F0410F4CD4F80880E7686569A679BB
:1023F000FFF7ECFF63792279E17943EA02220A4B85
:1024000001241C70094B0024EDB21C7003245C7085
:10241000C3F804809F601D735E73DA81197458617C
:10242000BDE8F081803F0008200300208C030020DD
:102430002DE9F04F054610F8013BDFF8F4C2A8493A
:10244000A84FDFF8F0A23B7089B0DA0901929DF83D
:1024500004208CF80020C3F380120A70C3F34012EA
:102460000092A14A04939DF80030CDF81CC005915C
:10247000137000F007FF6B1DCAF8000004461846F1
:10248000029300F0FFFEDFF8B0920390C9F800005D
:102490009648AA7902709648EE79067095482E7A89
:1024A000DFF8988295F805B0067005F109000692EC
:1024B00088F800B000F0E6FE8F4E306005F10D00A8
:1024C00000F0E0FE706005F1110000F0DBFE049BFF
:1024D0000199DDF81CC0B06003F01F033B70CDF81C
:1024E00010C0069A49B18548294605F1400E51F8B9
:1024F00004CB40F804CB7145F9D1013B0A2B00F223
:102500000D82DFE813F01F010B020B00690184014B
:10251000870148008D01B3010B02DF01784D2B7854
:10252000072B04D1774B1B785B4504D8F6E113B138
:102530000C2B40F0F381BBF1000F01D0FFF750FFEF
:10254000002398F800102B7018234B436E4A6F4EEF
:1025500012F803E0D4186E4B6E4A83F800E06378FB
:1025600003F0010111706C4AC3F3400313700FCCE8
:102570000FC694E8030086E80300BEF1000F02D006
:10258000BEF1010F02E000F07AFB012800F0C681E5
:1025900008232B7044E05A4B197801291E4600F29B
:1025A000BD810099DFF8988100293ED0D8F800302D
:1025B000002B40F08F80594B019283F800B0584BAC
:1025C000C8F80010E81D1C6000F05CFE554B019A35
:1025D0001860554B1A706FF0370303EB82023823F3
:1025E00003FB0424BBF1000F03D0BBF1010F05D0A6
:1025F00008E0464B9B689C4206D903E0434B1B7B9B
:102600009C420FD90A2366E0414B1B7813B1012B82
:1026100004D007E0FDF7D0FD012803D00823337074
:102620003A785AE00123337078E1D8F80010002995
:1026300050D03B4A1268944201D9032246E0013946
:102640008C4242D1013A94420ABF374B0E231B7889
:1026500000932F4B1C786CBB029D2046009BE2B27E
:102660009A4225D2284600F00DFE2C4AC9F80000F7
:102670001078FFF79BFEDAF800204FF0380B0BFBC9
:1026800002FB0BEB840B83440322002050B9584615
:10269000D9F800100192FEF743FC031F584258413D
:1026A000019A00E00120013AF0D101340435D5E768
:1026B000012804D0082333701C4B3A781A60D8F8EC
:1026C00000300133C8F8003028E102221A70174B9D
:1026D0001C6023E1082333700722144B1A601DE1AC
:1026E0001E0300201F03002023030020CA04002033
:1026F000CE040020CD0400207C0400208A040020A9
:1027000068030020200300208C03002074030020B5
:102710000F0500208904002088040020CB0400203D
:10272000C8020020CC02002021030020C4020020A7
:1027300022030020B802002070030020CC040020F7
:10274000C0020020FFF74CFE7E4B01221A700222CD
:102750005A7098F800201946CAB99A70DA701A713E
:102760005A719A71784B1C78CC711346A2420ADADE
:10277000764D182000FB025055004078A8400343D6
:102780009BB20132F2E71A0A0A724B721FE06F49DC
:102790009A71501E182404FB00114A7BDA710A7BDF
:1027A00088681A72CA8949695871050E0C0E9D70A5
:1027B0009C72050C0C0CDD70DC72050A0C0AD0B2A0
:1027C000120A1D7158721C7359739A73D8733F2182
:1027D0005F48FFF70BFDA1E0039A45F6FE239A42FE
:1027E00003D14FF6FF7000F039FD00203168FFF78C
:1027F0006DFD01207168FFF769FD0220B168FFF7E8
:1028000065FDFEF753FB534B01221A7086E0FDF77E
:1028100019FE83E0504A00231360504A13707DE094
:102820004E4C2378012B79D14B4D4D4A2B681168C2
:10283000013B8B4216460ED100232B60494B1B787F
:102840000BB1052306E0484B1F68FFF7BFFD874229
:10285000F7D00B2323702B683268013B93425DD283
:102860003D4B00221A600423237057E03B4B18783D
:10287000194618BB3D4B83F800B03D4B1C603D4BE7
:102880001A600E3A0E2303FB0424BBF1000F05D09F
:10289000BBF1010F09D1384B1A7B01E0364B9A6826
:1028A000944294BF0024012414B10A230B7007E062
:1028B000324B00221A6006230B702FE008221A7098
:1028C00009220AE71F4B2E4901221A700C225A7066
:1028D000224A10789871022815460CBF0A680968C8
:1028E0001B4801BF110E9970110CD97017BFC1F3AD
:1028F0000724110A0022DC7019714FF000045A718C
:102900004FF03F0118BF9A70DC711C725C72FFF7C8
:102910006DFC2B78052B04BF104B1C70049B1B789F
:10292000012B0CD11748059B1A784378134300F804
:10293000013F3F2109B0BDE8F04FFFF757BC09B098
:10294000BDE8F08F10050020200300208C0300203C
:1029500011050020DB020020C002002068030020D7
:10296000C8020020CB040020CC0200202403002059
:10297000D0020020BC02002074030020B40200201A
:10298000C40200208A0400202DE9F84F294F3B782B
:10299000062B4DD1284B294D294801221A700A22B5
:1029A0005A702A685A71110E9970110CD970110A57
:1029B0001971016801398A421C4604BF214B93F802
:1029C00000A0804618BF4FF00E0A4FF000095FFAD2
:1029D00089F3534518D22B684FEA89064FF0380B1C
:1029E0000BFB036B184B1878FFF7E0FC174B063610
:1029F0000BEB00011A78A01900F04FFC08B908236E
:102A00003B7009F10109E2E72B68D8F80020104873
:102A10000133013A93422B6081BF05233B700D4B7C
:102A20000A2288BF1A603F21BDE8F84FFFF7DEBBDE
:102A3000BDE8F88F68030020CF040020B402002016
:102A4000D0020020BC020020240300200F0500203B
:102A5000D0040020C4020020844641EA000313F0A1
:102A600003036DD1403A41D351F8043B40F8043B95
:102A700051F8043B40F8043B51F8043B40F8043B58
:102A800051F8043B40F8043B51F8043B40F8043B48
:102A900051F8043B40F8043B51F8043B40F8043B38
:102AA00051F8043B40F8043B51F8043B40F8043B28
:102AB00051F8043B40F8043B51F8043B40F8043B18
:102AC00051F8043B40F8043B51F8043B40F8043B08
:102AD00051F8043B40F8043B51F8043B40F8043BF8
:102AE00051F8043B40F8043B403ABDD2303211D398
:102AF00051F8043B40F8043B51F8043B40F8043BD8
:102B000051F8043B40F8043B51F8043B40F8043BC7
:102B1000103AEDD20C3205D351F8043B40F8043B97
:102B2000043AF9D2043208D0D2071CBF11F8013B95
:102B300000F8013B01D30B8803806046704700BF5B
:102B4000082A13D38B078DD010F003038AD0C3F16A
:102B50000403D21ADB071CBF11F8013B00F8013B4C
:102B600080D331F8023B20F8023B7BE7043AD9D30B
:102B7000013A11F8013B00F8013BF9D20B780370E0
:102B80004B7843708B7883706046704770B48407CD
:102B900046D0541E002A41D0CDB2034602E0621E48
:102BA000E4B3144603F8015B9A07F8D1032C2ED93D
:102BB000CDB245EA05250F2C45EA054519D903F1A3
:102BC00010022646103E0F2E42F8105C42F80C5CB4
:102BD00042F8085C42F8045C02F11002F2D8A4F159
:102BE000100222F00F0204F00F041032032C1344E1
:102BF0000DD91E462246043A032A46F8045BFAD849
:102C0000221F22F003020432134404F003042CB107
:102C1000C9B21C4403F8011BA342FBD170BC70472E
:102C200014460346C2E700BF08B540200121FEF765
:102C300079FB4FF080500121FEF78CFB4FF40050E0
:102C4000BDE80840FEF7CABB0120FEF7E9B9F8B5B8
:102C500005460F460024BD420DD25CB90326284626
:102C6000FEF740F9042802D0013EF8D1012405F511
:102C70000065F0E7012484F00100F8BD704708B555
:102C8000FEF706F9012008BD40200121FEF74ABBEE
:102C900010B504462CB14FF47A70FDF7CFFA013C21
:102CA000F8E7204610BD10B50446FDF7DFFA001B1B
:102CB00010BD00B9FEE703798B420FD901EB41014A
:102CC0000268CB00D118087D496818B1D05889B284
:102CD00000F0EEB8D05889B200F0E8B8704700B9FB
:102CE000FEE703798B420FD901EB41010268CB006B
:102CF000D118087D496818B1D05889B200F0D6B80B
:102D0000D05889B200F0D4B870470022531003F1B4
:102D10000053A3F6540312F0010F1B78DBB208BF77
:102D20001B0903F00F03092B8CBF372130210B4403
:102D300083540132182AE9D10023037618467047DC
:102D400008B5FDF755FC002814BF0320002008BD7E
:102D500030B5456985B0044615B304AA002302F8CE
:102D6000013D0092806904F15D013F22A8470546BC
:102D7000B0B1012384F85C3063689878FFF7A8F855
:102D80006A1C014692B204F15C0000F0A6F8636888
:102D900040219878FFF7BCF86368987800F019F93B
:102DA00005B030BD704721B9002814BF02200020B3
:102DB000704702207047FEE708B5FFF7FCFF08B533
:102DC000FFF7F9FF08B5FFF7F6FF08B5FFF7F3FFC8
:102DD00008B5FFF7F0FF08B5FFF7EDFF08B5FFF7FF
:102DE000EAFF08B5FFF7E7FF08B5FFF7E4FF01BE0C
:102DF000FEE710B50446FEF761F8012806D11CB1C4
:102E0000FEF75CF8013CF8E7052010BD002C08BF78
:102E1000052010BDF0B500230E681C460125A54015
:102E200005EA060EAE452BD10F797A1E012A15D878
:102E3000856803229A4025EA020282604D79826801
:102E40009D4015438560828892B222EA0E028280FC
:102E50008A798588A2402A4392B28280032205683B
:102E60009A40D2431540056005689F402F43076094
:102E7000C7681740CA7902FA03F547EA0502C2603B
:102E80000134102C03F10203C8D1F0BD4FF6FF73DB
:102E9000036002220023037142718371C371704782
:102EA000038A194214BF01200020704781617047D6
:102EB0000185704701F00703C90800EB810010B5D8
:102EC0009B00046A0F21994024EA01010162016A12
:102ED0009A401143016210BD704730B501F10051B5
:102EE000013201F54051521049000023934200F194
:102EF000020009D010F8015C10F8024C44EA0524E5
:102F000021F823400133F1E730BD10B501F1005144
:102F1000013201F54051521049000023934205D07F
:102F200051F8234020F813400133F7E710BD80002B
:102F300000F1804000F5B840036823F4EC4323F02F
:102F40007003194389B201607047800000F180402E
:102F500000F5B840CA06036823F4E04323F04003B9
:102F60009BB248BF83F010038A0648BF83F020035A
:102F700043F4004343F0800303607047800000F196
:102F8000804000F5B840CA04036823F4804323F06E
:102F900070039BB248BF83F480538A0448BF83F414
:102FA000005343F4004343F0800303607047800004
:102FB00000F1804000F5B840006800F03000704734
:102FC000800000F1804000F5B840006800F44050F7
:102FD0007047800000F1804000F5B840036823F49A
:102FE000E04323F040039BB283F0300343F40043FB
:102FF00043F0800303607047800000F1804000F5DB
:10300000B840036823F4804323F070039BB283F439
:10301000405343F4004343F0800303607047800053
:1030200000F1804000F5B840036823F4F8731B05F5
:103030001B0D43F4004343F080030360704780009E
:1030400000F1804000F5B84003685B0441BF0268AE
:1030500040F60F73134043F4404344BF43F08003F2
:1030600003607047800000F1804000F5B8400368BD
:103070005B0641BF026840F60F73134043F4004300
:1030800044BF43F0C00303607047C3B2000A40EA84
:103090000320704710B5B2FBF0F4B4FBF1F301FB71
:1030A00013434343B3FBF1F34143B2FBF1F1C907CF
:1030B00048BFC31A00FB1420984294BF002001208F
:1030C00010BD30B5054601B9FEE702B9FEE790F83C
:1030D0008700A0B13E2A12D905F1480205F184000B
:1030E00052F8044B41F8044B8242F9D11088088011
:1030F00092788A70002285F887203F2000E0002027
:1031000043B195F8872002F0FF0112B13F221A80E7
:1031100030BD198030BD30B5054690F8470000F04D
:10312000FF04A0B93E2A14D905F1080201F13C00C0
:1031300051F8044B42F8044B8142F9D108881080C1
:1031400089789170012285F847203F2002E0002015
:1031500000E0204633B195F847200AB93F2200E04D
:1031600000221A8030BD38B505460C4601B9FEE78D
:1031700002B9FEE73F2A06D0FEE76B68DB6813B1B1
:1031800028683F21984795F88730002BF5D12146D4
:1031900005F1480304F13C0251F8040B43F8040B19
:1031A0009142F9D10A881A808A789A70012385F8A9
:1031B00087306B68DB6813B128683F21984700208F
:1031C00038BD10B501B9FEE702B9FEE73F2A00D0CD
:1031D000FEE790F8473003F0FF0433B94368006816
:1031E0001B6911469847204610BD00F1080300F105
:1031F000440253F8044B41F8044B9342F9D11A8826
:103200000A809B788B70002380F847303F2010BDE8
:1032100008B5FFF709FDBDE80840FFF715BD10B57B
:103220000020FCF7B1FF04460120FCF7ADFF41F29E
:1032300022139C4205D14AF65523C31A58425841DD
:1032400010BD002010BD08B500200146FCF7AAFF04
:1032500001200021BDE80840FCF7A4BF0146022080
:10326000FCF7A0BF30B503460D466C1AE4B2944299
:10327000184603F1020304D215F8010B03F8020CFF
:10328000F3E730BD437802781B0403EB0263C27896
:103290008078134403EB00207047F8B505460F46CD
:1032A00062B9061D0446781B2044FFF7E7FC03784B
:1032B00004F8013BB442F6D10120F8BD0020F8BD6E
:1032C00000000000010000000200000003000000F8
:1032D00004000000050000000600000007000000D8
:1032E00008000000090000000A0000000B000000B8
:1032F0000C0000000D0000000E0000000F00000098
:10330000000000000000000000000000B9060008F6
:103310007106000841060008590600080000000078
:1033200000000000412D0008000000000000000027
:103330000000000000000000140C0001000000006C
:10334000000000000000000000000000000000007D
:10335000000400480002000001030000000000001B
:1033600000000000010000000004004820000000F0
:103370000103000000000000000000000100000048
:1033800000000048010000000103000000000000F0
:10339000000000000000000050330008030000009F
:1033A0000400050006002B424C0012035000690087
:1033B0006B006F00200042004C0058001C036F009F
:1033C000700065006E00700069006C006F00740092
:1033D0002E006F007200670004030904000101065B
:1033E0009CFF0901A10185010902150025FF75084F
:1033F000953F810385020902150025FF7508953F59
:103400009182C01201000200000040A020954101FD
:103410000B0102030109022900010100C07D09041A
:103420000000020300000009211001000122240015
:0E343000070581034000040705010340000466
:10344000D92E0008D92E0008D92E0008D92E000840
:10345000D92E0008D92E0008D92E0008D92E000830
:10346000D92E0008D92E0008D92E0008D92E000820
:10347000D92E0008D92E0008850B0008E10A0008A3
:10348000050A0008A52D0008190A0008C50B000848
:10349000A72D0008BD0A0008B10A0008910A00081B
:1034A0000000000040000000D92E0008A50B000815
:1034B000D92E0008D92E0008D92E0008D92E0008D0
:1034C000D92E0008D92E0008F909000800A24A04E4
:1034D00064000000640000008813000088130000EE
:1034E000010002000400060008000A000C001000A1
:1034F00020004000800000010000000000000000EB
:1035000001020100000000000000000102030406A7
:103510000708090000000001020304010203040679
:103520000708093803000000000000000000000048
:10353000000000000000000000000000000000008B
:10354000000000000000000000000000000000007B
:0C3550000000000000000000000000006F
:103F8000BDBDBDBD1005040100C000089C3F03007D
:103F90009CFF03086400000000400008008000004F
:103FA0000000000000000000000000000000000011
:103FB0000000000000000000000000000000000001
:103FC00000000000000000000000000000000000F1
:103FD00000000000000000000000000000000000E1
:103FE00000000000000000000000000000000000D1
:103FF00000000000000000000000000000000000C1
:0400000508000000EF
:00000001FF
